:020000040000FA
:06000000083004303A282C
:08000800A000030EA100831209
:1000100005191128831601178312B2308100B1012E
:100020002C2883160113831203140B190310A80D37
:10003000A90DAA0DAB0DAC0DAC16FF302C02031DA3
:100040002C28FA302B02031D2C2832152A08AF0069
:100050002908AE002808AD008B100B11210E83007B
:06006000A00E200E0900B5
:04006600003400342E
:0C007400203084008001840A6030040207
:10008000031C3C288F218316FF23900083128316C4
:100090000C3085058701831285018701073099009F
:1000A0000030831691009F008312C83083168100B0
:1000B000831231309000003083168C008312103090
:1000C0008B00BD1B6928851969286400851D65287A
:1000D000E521E02181018E018F010B118B100B10A6
:1000E0008C018B17812032198D20B40B7F280310CF
:1000F00085190314BA0DF0303A02031902210E22B9
:10010000722864003310B10A311F8C28AC01AB0196
:10011000AA01A901A801B101080032110130B700FC
:100120008B132030370783169B001C141A08831288
:10013000A4001030370783169B001C141A08831282
:10014000A300A6000230A6060030370783169B00E6
:100150001C141A088312A200A7000130A7068B17EF
:10016000331CB82822090339A200A309A409A50950
:1001700024082F02031DFC2823082E02031DD72864
:1001800022082D02031DFC2801303702031DCE2852
:10019000CD283E18CE283E143F14B221023037023B
:1001A000031DD728BE18D728BE143F14BA2126082D
:1001B0002E02031DF32827082D02031DFC28013001
:1001C0003702031DE928E8283E1CE9283E103F14A9
:1001D000BF2102303702031DF228BE1CF228BE10D8
:1001E0003F14C721FC285F08F039A03C0319FC2804
:1001F0002E1AFC28FB28CC21B70A0330370203183B
:10020000080090280130B600B400B500B7008501A1
:100210008701B213D92166218120B40B3329031041
:1002200085190314BA0DF0303A0203195B290C1C2E
:100230002A290C10C00A4208400203192829420A40
:1002400040020319662102303702031966212A2968
:1002500085018701B50B3329FA30B500023037022A
:1002600096300319B500321D0C293211331C3D297B
:100270002D090339AD00AE09AF092F1C0C292D083B
:10028000300203190C292D08B0002E1E0C298B13E7
:1002900020303707BC002F08BB007C211030370707
:1002A000BC002E08BB007C2100303707BC002D08A5
:1002B000BB007C218B1785018701DC21B70AB601C1
:1002C00003303702031C0C29E02108008E018F0146
:1002D000C0010C10013037020319CF210230370260
:1002E0000319D42108003F1C08003F101030BC0047
:1002F0003E08BB007C2108008B133B0883161C15AD
:100300009A003C089B0055309D00AA309D009C142B
:1003100064009C1888291C1183128B17080083160F
:1003200000309B001C141A088312BD008316103085
:100330009B001C141A088312BE00831620309B00F9
:100340001C141A088312C2000130C21BC200C2086A
:100350000319C200831630309B001C141A08831244
:10036000DF0008000512051440084207D0004108CC
:10037000D10008000130CC000130C8000800051091
:10038000051640084207D0004108D100080002309D
:10039000CC000130C800080005100512080038091B
:1003A00011398500B8000800380922398500B800E5
:1003B0000800B80138140800B801B814B8160800CD
:1003C000BE18BA21BE1CC7210800B601B401B50190
:1003D0003D1CED29BD01BD14EF29BD013D143D08B3
:1003E000B6006400F329F429F529F629F729B51B8D
:1003F0008514B51F8510B51B8516B51F8512B40B66
:10040000F129B50BF1290310B60CB608031DF1292B
:100410000030BC003D08BB007C2108008F08031998
:1004200008008F013C308E004D094C05CA004C0974
:100430004D05CB00C8080319232AFF303D1CC80016
:10044000C80F362A5922C10A0319C00A5F080F399A
:100450000A3C0319080050084002031D0800510817
:100460004102031C08000510051208004808C900D5
:100470004A188514CA18851649080E020318482A16
:100480004B188510CB188512FF304802031908005D
:100490008F08031D0800812049080E02031C482A0A
:1004A0004A188510CA1885124B188514CB18851662
:1004B00008004A188514CA188516CA014B188510F9
:0E04C000CB188512CB014C08CD00732108002B
:084000000A000300060009009C
:02400E00CC01E3
:10420000010078007A007C007E007B0079007F004E
:104210007D007A0078007E007C00FF00FF00FF0038
:104220000000F200F600FA00FE00F200F600FA00CC
:10423000FE00F200F600FA00FE00FF00FF00FF00A3
:10424000010005000500050005000900090009003E
:1042500009000D000D000D000D00FF00FF00FF0024
:10426000FF00FF00FF00FF00FF00FF00FF00FF0056
:10427000FF00FF00FF00FF00FF00FF00FF00FF0046
:10428000FF00FF00FF00FF00FF00FF00FF00FF0036
:10429000FF00FF00FF00FF00FF00FF00FF00FF0026
:1042A000FF00FF00FF00FF00FF00FF00FF00FF0016
:1042B000FF00FF00FF00FF00FF00FF00FF00FF0006
:1042C000FF00FF00FF00FF00FF00FF00FF00FF00F6
:1042D000FF00FF00FF00FF00FF00FF00FF00FF00E6
:1042E000FF00FF00FF00FF00FF00FF00FF00FF00D6
:1042F000FF00FF00FF00FF00FF00FF00FF00DD00E8
:00000001FF
